:04000000020029329F
:01000B0032C2
:0100130032BA
:01001B0032B2
:030023000203D500
:0300850002002650
:030026000200884D
:200088007F01C0071203AC75C70F1204CAD007E5B00303540FF4FEEF4206EEC454F0FE74BF
:2000A8000F4EF5C77D007E007B007C00C007C006C005C004C0031204FBE582D003D004D065
:2000C80005D006D007601AC007C006C005C004C00312050E1204EBD003D004D005D006D0CB
:2000E800070BBB00010CEC60C30DBD00010EC3ED9440EE940040B1EF2FFF24F050917F01AD
:040108000200972238
:03008200750B00FB
:20010C002290FBC0E493FCA3E493FDA3E493FEA3E493FFBCF011BD1D0EBEAD0BBFB0089089
:20012C00FBC075F08080517E007F0EC3E49E74FA9F503F8E828F83E493FAA3E493FBA3E427
:20014C0093FCA3E493FDBAF017BB1D14BCAD11BDB00E8E038F047D808B828C838DF08018F9
:20016C008E048F05EC24C0FCED34FFFD8C068D0780B990000075F00022901B0075F0B7E443
:20018C002285820AC2CAE50A700302022C120185AB82AC83ADF0FEE50A75F004A42408F556
:2001AC0082740635F0F583E493F8A3E493F9A3E493FAA3E4938A18C42354E0C518C423C5A4
:2001CC00186518C51854E0C5186518F519E9C423541F4518F5188816E9C42354E0C516C417
:2001EC0023C5166516C51654E0C5166516F5178B828C838DF0EE1205B2AC82AD83AEF0FFBE
:20020C00E4C39CFCE49DFD74019EE49F8C067F008ECA8D047D008CCB85CACC85CBCDD2CADD
:20022C00850A082222AF82A2AF9200C2AFE5B054306002800ABF08028003BF18027F07E4BE
:20024C00BF180104FE7003BF084875B167EE60047E1080027E00EE42B1AEB274F85E440476
:20026C00F5B27DB87E0B1DBDFF011EED4E70F7FDFEC3ED94B8EE6480948B5011748055B130
:20028C00FCBC800280070DBD00E70E80E475B20C8040AEB25306F88F05ED4EF5B27DB87EA1
:2002AC000B1DBDFF011EED4E70F7FDFEC3ED94B8EE6480948B5011741055B2FCBC1002806F
:2002CC00070DBD00E70E80E4AEB274F75EF5B275B107A20092AF7D007E007B007C00EB2407
:2002EC0040F582EC3406F583E493FAB507028D0974052BFBE43CFC0DBD00010EC3ED9406FA
:20030C00EE6480948040D722AF82AEA4D2017D0074F02DF5A48D037C0074F02BFBE43CFC03
:20032C00A9A47A00E9B50306EAB504028004C20180060DBD100040D83001028EA4AE97D263
:20034C00027D0074F02DF5978D037C0074F02BFBE43CFCA9977A00E9B50306EAB5040280BD
:20036C0004C20280060DBD100040D83002028E97300205750B018027200105750B02801F32
:20038C00750B03E5B0541C7007C00712E000D007C00712023012010CD0078F821202312249
:2003AC00AFD974BF5FF5D975D90075F2DF75A43175AEF075D52075E10975E24075B2C37599
:0903CC008920758E01758D6422F3
:20060800000000006E000000960000002C01000058020000B004000060090000C012000058
:2006280080250000004B00000096000000E1000000C20100000000000480841E0005000954
:160648003D000600127A00070024F4001800C0A800080080510154
:2003D500C0E0C007C000C0D075D000309818E515045407FFB514028009E515240CF8A6991F
:2003F5008F15C2988007309904D203C299D0D0D000D007D0E032AC82AD83AEF0FF751400B9
:20041500751500D203200313C007C006C005C00412052ED004D005D006D007759840D2ACB6
:20043500D29C7597F07455F597B597051204A3805CC2C9C2C88C168D178E188F1990460083
:2004550075F005E41205B2AC82AD83AEF0FF8C03C3E49BFB8BCA8BCCE4C39CFCE49DFD74CC
:20047500019EFEE49FFFE4F516751701F518F5198C828D838EF0EF1205B2AC82AD83AEF061
:20049500FF8CCB8CCDD2CDD2CCD2CAD2AF22751400751500D203740F55894420F589758DEF
:2004B500FD758BFD53877FC2AB759840D2ACD29CD28ED2AF22751400751500D203740F556B
:2004D500892420F58953877FC2AB759840D2ACD29CD28ED2AF22AF823003FD8F99C2038FDD
:2004F50082221204EB22E514B5150474018001E4FFB40100E433F582221204FBE58260F94A
:20051500C2ACAF140514EF240CF98782531407D2AC2212050E1204EB22900000E4F5F0129A
:18053500040B1204A37582001204EB1204FB7582001204F71205272279
:20054D00FB7A20E4FCFDFEFFE5822582F582E58333F583E5F033F5F0EB33FB4017DAE980E7
:20056D0042E5822582F582E58333F583E5F033F5F0EB33FBEC33FCED33FDEE33FEEF33FF16
:20058D00EC9516ED9517EE9518EF95194013EC9516FCED9517FDEE9518FEEF9519FF438270
:0505AD0001DABEEB22A3
:06005800E478FFF6D8FD7C
:200036007900E94400601B7A0090065E780075A000E493F2A308B8000205A0D9F4DAF2750D
:02005600A0FF09
:20005E007800E84400600A790075A000E4F309D8FC7800E84400600C7900900000E4F0A3A2
:04007E00D8FCD9FAD7
:2005B200FBC2D530E715D2D5E4C39582F582E49583F583E495F0F5F0E49BFBE51930E71727
:2005D200B2D5E4C39516F516E49517F517E49518F518E49519F519EB12054D30D513FBE405
:1205F200C39582F582E49583F583E495F0F5F0E49B2243
:0D002900758120120604E5826003020026A6
:0406040075820022D9
:00000001FF
